:1000000000308A003A280000831A0A28A500030E4F
:10001000A6000F288312A500030EA600A6140A0846
:10002000AD008A018313A50E0408A7002008A800CC
:100030002108A9002208AA002308AB002408AC006C
:1000400083120B1E25288B185428270884002808A3
:10005000A0002908A1002A08A2002B08A3002C0850
:10006000A4002D088A00260E83008312250EA618F0
:1000700083160900FF238316900000308A00502A5F
:10008000513084000008031953280130A100A00159
:10009000A00B4828A10B47284A30A000A00B4E28EF
:1000A0005128800B452800340B1283160515831246
:1000B000051962283230D100402083160512103015
:1000C000831285068B108A112528C0014008073C41
:1000D000031C842883168512831285126F2803104F
:1000E000BF0C03187528851276288516831685128D
:1000F00013308312A000A00B7B287E288316851660
:1001000081288312C00A6628003483168512831260
:100110008512A630A000A00B8B2800008316851640
:10012000A6308312A000A00B93280000831685162A
:1001300083120034BF013F08073C031CBC28831610
:10014000851283128512A428831685160230831225
:10015000A000A00BA9280000831685168312851A1B
:10016000B3280310B4280314C00C2730A000A00B40
:10017000B728BA28BF0A9B284008A1000034B6015E
:100180008520CC30BF0065204430BF006520AE0123
:100190008B1BAE178B13C830D1004020AE1B8B17C2
:1001A000B608031DD7289A202108B600D02885203C
:1001B000CC30BF006520BE30BF0065209A202108EA
:1001C000B7009A202108B8009A202108AF009A2091
:1001D0002108B0009A202108B1003808BA00370879
:1001E000B9003A08C0003908BF008E30A0004008AE
:1001F000A1003F08A200A301C01F0329A109A20971
:10020000A20A0319A10AA108031D10292208A100AE
:10021000A2010830A002A108031D1029A00119297C
:100220000310A11B1729A20DA10DA0031029C01FA7
:10023000A1132008BF002108C0002208C100230824
:10024000C2004208C6004108C5004008C4003F087B
:10025000C300CA01C901C8018330C700430803199C
:10026000F329CF0047080319F329CF02031C3D29C6
:100270007F30CF070318F32943298130CF02031CB5
:10028000F3290319F3294F08A000A101A201A3013A
:10029000CE014408CD00CD174508CC004608CB0060
:1002A0001930CF004A08CB02031866290130CC026E
:1002B00003186629CD0203186629CE0203186629A1
:1002C000CE0ACD0ACC0A4A08CB0798294908CC02A5
:1002D000031881290130CD0203188129CE020318A9
:1002E0008129CE0ACD0A4908CC074A08CB07031C4E
:1002F0009829CC0A031D9829CD0A031D9829CE0AF6
:10030000982948088038CD02031897290130CE0279
:1003100003189729CE0A48088038CD074908CC072A
:10032000031C7529CD0A031D7529CE0A75292314CE
:10033000CF0B9B29A6290310CB0DCC0DCD0DCE0DD7
:100340000310A30DA20DA10DD00D5229501CAE29F2
:100350000310A10CA20CA30CD00CB129A00303190B
:10036000F329D01BDA290310CB0DCC0DCD0DCE0D0A
:100370004A08CB020318C6290130CC020318C6294B
:10038000CD020318C629CE02031CE9294908CC0274
:100390000318D1290130CD020318D129CE02031C44
:1003A000E92948088038CD020318DA290130CE0245
:1003B000031CE929A30A031DE929A20A031DE9294F
:1003C000A10A031DE929A00A0319F329A10CA20C13
:1003D000A30C4408CF004808CF06CF1FF129A1176E
:1003E000F729A113F729A001A101A201A301230864
:1003F000BE002208BD002108BC002008BB00AE01E1
:100400008B1BAE178B13C830D1004020AE1B8B174F
:100410003B08A0003C08A1003D08A2003E08A30044
:100420008F2A3708BE003B08BE06BE1F1C2A0311D8
:100430000310B71B03144F2A3708BE003A08BF0049
:100440003608BF0203192A2ABE1F4F2A0308013AA1
:1004500083004F2A3B08BF003708BF020319362A22
:10046000BE1F4F2A0308013A83004F2A3C08BF00F1
:100470003808BF020319422ABE1F4F2A0308013A57
:1004800083004F2A3D08BF003908BF0203194E2AD6
:10049000BE1F4F2A0308013A83004F2A031000347D
:1004A00003081F3983003F30A000213084008313EC
:1004B0008001840AA00B582AA00184011F30830503
:1004C0000730990083160108C73908388100831264
:1004D0009001CC30BF0065204E30BF0065207D30DC
:1004E000BF006520C930BF0065207F30BF00652098
:1004F0008520CC30BF0065204830BF006520AE01AC
:100500008B1BAE178B130F30D1004020AE1B8B1707
:100510000B1683160113C03083128B04BF282308E7
:10052000B5002208B4002108B3002008B200350845
:10053000B9003408B8003308B7003208B600BD016E
:10054000BC012030BB008430BA001122031CB12A48
:1005500083160510831205148316851083128510E7
:10056000B92A831685108312851483160510831209
:100570000514B901B8010C30B7008530B600350854
:10058000BD003408BC003308BB003208BA00112299
:10059000031CDB2A8316851083128514831605102D
:1005A000831205108316851583128519DB2A83169D
:0A05B000051283120512882A630069
:02400E0014316B
:00000001FF
